:100000000C94D6040C941D050C941D050C941D0530
:100010000C941D050C941D050C941D050C941D05D8
:100020000C941D050C941D050C941D050C94580D85
:100030000C94070E0C94C01B0C941D050C941D050C
:100040000C941D050C941D050C941D050C94341C7A
:100050000C941D050C941D050C941D050C941D0598
:100060000C941D050C941D050C941D050C941D0588
:100070000C941D05740E960E840F960E840FDB0EE5
:10008000FE0E840F530F660FA012A012CD12CD12D8
:10009000281364135C155C157C135C1577147714B6
:1000A00032155C155C154815041607090B0A1D1B53
:1000B00006198005141A08151C171E1F202123225B
:1000C0002E26242D25273012182F0C13280F0D341F
:1000D0000E333136381110372B2C352A7F80807B38
:1000E00079397A808080808080634F80808050530F
:1000F0005180808058525780808062595A5B5C5D85
:100100005E5F8060618080808080568080806680B5
:1001100054808080805580800A0025303862003A03
:10012000200025303258000A722F632030313233DC
:10013000343536370A005D0A0025303258005B003E
:10014000200025303258002831290A002832290A97
:10015000002833290A002834290A000A00253032F1
:1001600058006D303131305F726563762065727290
:100170003A20000A0025303258006D303131305FAE
:1001800073656E64206572723A20005B735D004B8C
:100190006579626F6172642073746172742E0A00F3
:1001A00055534220636F6E666967757265642E0AE7
:1001B000005B575D005B535D005B525D0032034D99
:1001C00000300031003100300020006B0065007904
:1001D0000062006F00610072006400200063006F25
:1001E000006E007600650072007400650072000009
:1001F000000E0374002E006D002E006B002E000018
:10020000000403090409027400040100A032090477
:100210000000010301010009211101000122400039
:100220000705810308000A09040100010301020017
:10023000092111010001224D000705820308000A6F
:10024000090402000103000000092111010001223C
:1002500036000705830308000A09040300020300AF
:10026000000009211101000122220007058403205A
:100270000001070504032000011201100100000025
:1002800008EDFE10010101010200010631FF0974B1
:10029000A1010975150026FF009520750881020946
:1002A00076150026FF00952075089102C00501090A
:1002B00080A101850216810026B7001A81002AB7A5
:1002C00000751095018100C0050C0901A10185038D
:1002D000160100269C021A01002A9C027510950145
:1002E0008100C005010902A1010901A10005091948
:1002F00001290515002501950575018102950175F6
:100300000381010501093009311581257F950275A9
:1003100008810609381581257F9501750881060534
:100320000C0A38021581257F950175088106C0C029
:1003300005010906A101050719E029E715002501B6
:10034000950875018102950175088101050819015B
:100350002905950575019102950175039101050720
:10036000190029FF150026FF00950675088100C0B9
:100370000A002530325820006B6579626F61726423
:100380005F7265706F72743A20004C45443A2025C4
:100390003032580A00290A002575002F0025750003
:1003A0005D280025640020002564002000256400ED
:1003B00020002564007C0025303258006D6F757375
:1003C000656B6579205B62746E7C7820792076207D
:1003D000685D287265702F61636C293A205B006D3F
:1003E0006B5F776865656C5F74696D655F746F5F7F
:1003F0006D6178203D2025640A006D6B5F7768652C
:10040000656C5F6D61785F7370656564203D202564
:10041000640A006D6B5F74696D655F746F5F6D6119
:1004200078203D2025640A006D6B5F6D61785F73F5
:1004300070656564203D2025640A006D6B5F696E00
:1004400074657276616C203D2025640A006D6B5FD7
:1004500064656C6179203D2025640A006D6B5F77CF
:100460006865656C5F74696D655F746F5F6D6178F9
:10047000203D2025640A006D6B5F776865656C5FC1
:100480006D61785F7370656564203D2025640A00A6
:100490006D6B5F74696D655F746F5F6D6178203D32
:1004A0002025640A006D6B5F6D61785F7370656510
:1004B00064203D2025640A006D6B5F696E7465726F
:1004C00076616C203D2025640A006D6B5F64656C6D
:1004D0006179203D2025640A000A00257500363A1E
:1004E00020776865656C5F74696D655F746F5F6DBB
:1004F00061783A20000A00257500353A2077686552
:10050000656C5F6D61785F73706565643A20000AA1
:1005100000257500343A2074696D655F746F5F6DF6
:1005200061783A20000A00257500333A206D617821
:100530005F73706565643A20000A00257500323AE1
:1005400020696E74657276616C286D73293A20009B
:100550000A00257500313A2064656C6179282A31DA
:10056000306D73293A20000A092D2056616C75659B
:1005700073202D0A004D3E004D25643E20003F00B3
:100580007365742064656661756C740A00433E206F
:100590000077686572652064656C74613A206375E4
:1005A00072736F723D25642C20776865656C3D25FC
:1005B000640A53656520687474703A2F2F656E2E37
:1005C00077696B6970656469612E6F72672F7769EF
:1005D0006B692F4D6F7573655F6B6579730A000AE0
:1005E000092D204D6F7573656B6579202D0A455374
:1005F000432F713A09717569740A313A0964656C5F
:100600006179282A31306D73290A323A09696E748A
:10061000657276616C286D73290A333A096D6178C9
:100620005F73706565640A343A0974696D655F7457
:100630006F5F6D61780A353A09776865656C5F6D43
:1006400061785F73706565640A363A097768656535
:100650006C5F74696D655F746F5F6D61780A0A70B5
:100660003A097072696E742076616C7565730A64FC
:100670003A097365742064656661756C74730A75F4
:10068000703A092B310A646F776E3A092D310A707E
:100690006775703A092B31300A7067646F776E3A6C
:1006A000092D31300A0A7370656564203D20646548
:1006B0006C7461202A206D61785F737065656420B9
:1006C0002A2028726570656174202F2074696D6519
:1006D0005F746F5F6D6178290A003F004D3E200016
:1006E000433E20004C25640A000A092D20436F6E0A
:1006F000736F6C65202D0A4553432F713A0971754C
:1007000069740A6D3A096D6F7573656B65790A00D6
:100710000A092D204D61676963202D0A643A096436
:10072000656275670A783A096465627567206D616C
:10073000747269780A6B3A096465627567206B6543
:1007400079626F6172640A6D3A0964656275672047
:100750006D6F7573650A763A0976657273696F6EA7
:100760000A733A097374617475730A633A09636FA3
:100770006E736F6C65206D6F64650A302D343A09B5
:100780006C61796572302D34284631302D4634291C
:100790000A506175733A09626F6F746C6F616465BA
:1007A000720A003F0074696D65725F72656164333F
:1007B0003228293A202530346C580A006B6579625A
:1007C0006F6172645F69646C653A2025580A006B3A
:1007D0006579626F6172645F70726F746F636F6C62
:1007E0003A2025580A00686F73745F6B6579626FF1
:1007F0006172645F6C65647328293A2025580A0089
:100800000A092D20537461747573202D0A00474323
:10081000433A20342E392E32204156522D4C494233
:10082000433A20312E382E3073766E204156525F77
:10083000415243483A2061767233350A004F505492
:10084000494F4E533A204C554641204D4F55534544
:100850004B45592045585452414B455920434F4E22
:10086000534F4C4520434F4D4D414E44204B45592D
:100870004D41505F53454354494F4E203430393633
:100880000A004255494C443A206337666435666332
:100890002D6469727479202830343A31393A31390B
:1008A000205365702031332032303136290A00560A
:1008B00049443A2030784645454428742E6D2E6BC5
:1008C0002E29205049443A20307830313130284D9B
:1008D00030313130206B6579626F61726420636FF3
:1008E0006E76657274657229205645523A203078CA
:1008F000303130310A00444553433A20636F6E76FD
:10090000657274204D30313130206B6579626F61D2
:10091000726420746F205553420A000A092D205634
:10092000657273696F6E202D0A000A6D6F757365AD
:100930003A206F66660A000A6D6F7573653A206F1C
:100940006E0A000A6B6579626F6172643A206F66A5
:10095000660A000A6B6579626F6172643A206F6E95
:100960000A000A6D61747269783A206F66660A003F
:100970000A6D61747269783A206F6E0A000A6465C4
:100980006275673A206F6E0A000A64656275673A9D
:10099000206F66660A000A0A626F6F746C6F61648A
:1009A00065722E2E2E2000433E20000011241FBE13
:1009B000CFEFD4E0DEBFCDBF04B603FE27C08091E9
:1009C000D4019091D501A091D601B091D701873083
:1009D000904BA740B04BD1F41092D4011092D501A6
:1009E0001092D6011092D70114BE84B7877F84BFBE
:1009F0000FB6F894A895809160008861809360009C
:100A0000109260000FBEE0E0F8E3099511E0A0E06D
:100A1000B1E0E4E9F9E402C005900D92A233B10718
:100A2000D9F721E0A2E3B1E001C01D92A43DB207D5
:100A3000E1F70E94A50A0C94C8240C940000FF93CF
:100A4000EF93E0913201F0913301309709F009956D
:100A5000EF91FF910895FC018591803011F0EFDF57
:100A6000FBCF0895FF27E0E230E247FF0CC041953D
:100A700097FF09C0EDE26095709580959095611D96
:100A8000711D811D911D27FF02C0219530E350E2A9
:100A9000AA27660F771F881F991FAA1FA41710F097
:100AA000A41B63955A95A9F7AA3008F0A95FA05D29
:100AB000AF93F395611571058105910541F7ED320D
:100AC00011F4EF93F395F21718F43F93F395FBCFDE
:100AD0008F91B5DFFA95E1F70895E991F991859144
:100AE000803021F0853219F0AADFF9CF089520E097
:100AF000E89455915532C1F3503311F468945591EF
:100B00005A3348F4505390F3220F022E220F220F33
:100B1000200D250FF4CF0EF421958991999153362C
:100B200019F3533729F1533559F1BC018827992717
:100B3000E8945C3621F489919991689455915436E2
:100B400039F446EF7EF077FF0DC08FEF9FEF0AC0BC
:100B500055374AE039F0583540E121F0523642E04D
:100B600009F00895FF93EF937DDFEF91FF91B7CFE9
:100B7000FF93EF93FC0181918030B9F360DFFBCFED
:100B8000FF93EF9368DFF1CFDF93CF93CDB7DEB75D
:100B90002596A3DFCF91DF9108950E94C206E4E37A
:100BA000F1E08EE08E0F11928E13FDCF84E391E081
:100BB0009093430180934201569A5E9A2FEF89E603
:100BC00098E1215080409040E1F700C00000569A23
:100BD0005E980895CF93109244010E94DC07C82FBD
:100BE0008B3709F444C08F3F09F441C081E0809302
:100BF00044018C2F869586958695E0914201F0916F
:100C000043014C2F4770C7FF0EC08F70E80FF11DD6
:100C100021E030E001C0220F4A95EAF7209580815B
:100C2000282320830BC0E80FF11D81E090E001C074
:100C3000880F4A95EAF79081892B80838091B601CD
:100C400080FF17C08EE391E00E942B051F92CF9387
:100C500089E391E09F938F930E94C40586E391E01E
:100C60000E942B050F900F900F900F9002C080E014
:100C700001C081E0CF91089520914201309143015C
:100C8000F901E80FF11D80810895EF92FF920F9313
:100C90001F93CF93DF9387E291E00E942B05C0E082
:100CA000D0E082E2E82E81E0F82E0AE111E0DF9345
:100CB000CF93FF92EF920E94C4058FE191E00E94D2
:100CC0002B05E0914201F0914301EC0FFD1F808163
:100CD0000E94591B1F928F931F930F930E94C4056C
:100CE00088E191E00E942B0521968DB79EB708966A
:100CF0000FB6F8949EBF0FBE8DBFCE30D105B9F6AA
:100D0000DF91CF911F910F91FF90EF900895569A28
:100D100081FF02C05E9A08955E9808955198599A8D
:100D200008955898509A08955098589A089551984F
:100D3000599A85E08A95F1F7000089B1869581700E
:100D40000895CF93DF93EC010E949706882341F02A
:100D5000209731F085E08A95F1F700002197F4CFD4
:100D6000CE01DF91CF9108958B3741F08F3F41F055
:100D7000982F9F7796958078892B08958BE7089513
:100D80008FEF08950E948E060E9494062FEF83ED48
:100D900090E3215080409040E1F700C000000895AA
:100DA000EF92FF920F931F93CF93DF93E82E109251
:100DB00048010E948E060E949106CAEFD0E088EE9C
:100DC00093E00E94A106892B21F42197C1F781E0CD
:100DD00036C008E010E080E8F82E8AEF90E00E942C
:100DE000A106892B11F483E02AC08F2D8E2129F0D2
:100DF0000E949406C8ECD0E00AC00E949106FACF87
:100E0000209759F025E02A95F1F7000021970E94DC
:100E100097068823A9F3CD2B11F484E010C0F69433
:100E200001501109D1F68FE891E00197F1F700C068
:100E300000000E948E060E94940681E026C08093E6
:100E400048018AE791E00E942B05809148011F929A
:100E50008F9385E791E09F938F930E94C40583E76A
:100E600091E00E942B059FEF29E688E191502040F8
:100E70008040E1F700C000000E948E060E949406A8
:100E80000F900F900F900F9080E0DF91CF911F9106
:100E90000F91FF90EF9008950F931F93CF93DF93DF
:100EA00010924801CAEFD0E088EE93E00E94A106BC
:100EB000892B21F42197C1F781E02FC0D8E0C0E051
:100EC000CC0F88EC90E00E94A106892B11F482E0FF
:100ED00024C008EC10E00E94970681110AC0011599
:100EE000110549F025E02A95F1F70000015011099C
:100EF000F2CF012B11F483E010C05098589A85E08E
:100F00008A95F1F700004899C160D150C9F60E9456
:100F10008E060E9494068C2F26C08093480182E69C
:100F200091E00E942B05809148011F928F938DE5DF
:100F300091E09F938F930E94C4058BE591E00E94FE
:100F40002B059FEF29E688E1915020408040E1F792
:100F500000C000000E948E060E9494060F900F9021
:100F60000F900F908FEFDF91CF911F910F91089508
:100F7000CF9384E10E94D0060E944C07C82F8B3784
:100F8000C1F08091B60180FF0CC01F92CF9382E424
:100F900091E09F938F930E94C4050F900F900F9044
:100FA0000F908091B60180FF04C080E491E00E9420
:100FB0002B058C2FCF910895CF93DF93809147011C
:100FC000882319F0109247017EC080914601882342
:100FD00019F01092460177C0C0914501CC2319F059
:100FE0001092450103C00E94B807C82F8C2F8F773D
:100FF0008137B1F0893709F061C00E94B807982F96
:101000009F779D3041F018F4953039F404C0913148
:1010100011F09B3111F487FD37C00E94B4063AC02D
:101020000E94B807982F9F77913719F0993721F0D0
:1010300041C08093450142C00E94B807D82F8F77E6
:101040008D3041F018F4853081F504C0813111F004
:101050008B3159F5C7FF11C0D7FF0AC086E591E073
:101060000E942B058C2F0E94B406809346010BC072
:1010700081E591E00E942B0521C0D7FF0DC08CE4D3
:1010800091E00E942B058D2F0E94B406982F906648
:1010900090934701806417C087E491E00E942B057C
:1010A0008D2F0E94B40680660EC08D2F0E94B4065C
:1010B000806402C00E94B406809347018C2FDF91A8
:1010C000CF910C94B406DF91CF9108958091540193
:1010D00008959FB7F89410924B019FBF9091CB0158
:1010E000943009F057C09091E9009F703091EC0066
:1010F000232F217030FD20E8922B24E02093E9007B
:101100002091EB0020FF43C02091EE0027FF3FC05D
:1011100020914901222321F02091E80025FF37C0CA
:101120001092490126E03091E80035FD15C030915C
:10113000CB01343061F53091EB0035FD28C02150F2
:1011400021F481E08093490122C0EFE9FFE031976B
:10115000F1F700C00000E7CF8093F1008091E80034
:1011600085FD0AC08091E80080FFFCCF8091E800F7
:101170008E778093E80006C08FB7F89421E0209323
:101180004B018FBF9F709093E90080E008959F709E
:101190009093E9008FEF0895CF93DF9300D01F92D3
:1011A000CDB7DEB79C018091CB01843019F593E077
:1011B00099833B832A839093E9008FEF9091E80015
:1011C000815095FD06C095ED9A95F1F700008111CB
:1011D000F5CF8091E80085FF0DC040E050E063E06E
:1011E00070E0CE0101960E94660B8091E8008E7738
:1011F0008093E8000F900F900F90DF91CF910895AA
:10120000CF93DF9300D01F92CDB7DEB72091CB01F3
:10121000243021F522E029839B838A8383E0809315
:10122000E9008FEF9091E800815095FD06C095EDA3
:101230009A95F1F700008111F5CF8091E80085FFC4
:101240000DC040E050E063E070E0CE0101960E94E6
:10125000660B8091E8008E778093E8000F900F90E6
:101260000F90DF91CF9108952091CB012430F1F4BC
:1012700022E02093E9002FEF3091E800215035FD66
:1012800006C035ED3A95F1F700002111F5CF209118
:10129000E80025FF0BC040E050E065E070E00E94F0
:1012A000660B8091E8008E778093E8000895CF93D5
:1012B000DF932091CB01243039F521E02093E90020
:1012C0002FEF3091E800215035FD06C035ED3A95FD
:1012D000F1F700002111F5CF2091E80025FF14C09F
:1012E000EC0140E050E068E070E00E94660B809105
:1012F000E8008E778093E80088E0FE01ACE4B1E07E
:1013000001900D928A95E1F7DF91CF91089589EBD5
:1013100091E00C942B0520914A012F5F822F62E30C
:101320000E948E24992319F020934A010895109267
:101330004A0180914B01882371F18091CB01843067
:1013400041F58091E9008F702091EC00922F91700F
:1013500020FD90E8892B94E09093E9009091EB00B8
:1013600090FF14C09091EE0097FF10C09091E8009C
:1013700095FF03C01092F100F9CF9091E80090FF23
:1013800005C09091E8009E779093E8008F7080935D
:10139000E90010924B01089542E061EC81E00E9467
:1013A0006F0C42E061EC82E00E946F0C42E061EC65
:1013B00083E00E946F0C42E261EC84E00C946F0CBD
:1013C0008091CD01833009F453C030F4813071F045
:1013D000823009F48CC008958A3009F478C08B30CB
:1013E00009F45EC0893009F09AC020C08091CC0118
:1013F000813A09F094C08091E800877F8093E800EB
:101400008091D0019091D101892B21F468E08CE486
:1014100091E003C060E080E090E070E00E94B10BDA
:101420008091E8008B778093E80008958091CC014B
:10143000813209F074C08091D0019091D101892B43
:1014400009F06DC08091E800877F8093E80080916B
:10145000E80082FD05C08091CB018111F8CF5FC00B
:101460008091F100809354018091E8008B7753C004
:101470008091CC01813A09F052C08091D0019091C5
:10148000D101892B09F04BC08091E800877F8093C0
:10149000E8008091E80080FFFCCF80910A0136C00F
:1014A0008091CC018132D9F58091D0019091D10108
:1014B000892BA9F58091E800877F8093E8000E943E
:1014C000A40C8091CE0180930A010C947D1580912B
:1014D000CC01813221F58091E800877F8093E8007C
:1014E0000E94A40C8091CF018093550108958091B2
:1014F000CC01813AA1F48091E800877F8093E800D5
:101500008091E80080FFFCCF809155018093F1002D
:101510008091E8008E778093E8000C94A40C0895E5
:1015200008950895089585EB91E00E942B050C9491
:10153000920A0E947F1B8091C901882329F00E9492
:10154000AA1B81110C94500B089584B7877F84BF28
:101550000FB6F894A8958091600088618093600030
:10156000109260000FBE90E080E80FB6F894809370
:101570006100909361000FBE0E94900A0E942E109D
:101580000E94F50C0E94480D8091E20084608093D7
:10159000E20089E698E00E94541B78948091CB0188
:1015A0008430E1F780EA91E00E942B050E94301020
:1015B00080E091E00E949C0F8FE891E00E942B0553
:1015C0000E94910A8091CB01853039F48BE891E03B
:1015D0000E942B050E94990AF5CF0E943410F2CF89
:1015E0000C94BE1B81EB91E00E942B050C94F00A39
:1015F000292F332723303105C9F064F42130310518
:1016000081F02230310509F043C084E790E025E005
:1016100032E042C021323105F1F02232310541F190
:1016200037C082E190E029E732E036C09927813067
:10163000910541F08230910541F0892B49F5E1E0B7
:10164000F2E005C0E1EFF1E002C0EDEBF1E08491E2
:1016500090E09F0121C06430D8F4E62FF0E0EE0F57
:10166000FF1FE15EFE4F2081318189E090E014C0D0
:10167000643070F470E0FB01EE0FFF1FE95EFE4F77
:1016800020813181FB01ED5EFE4F808190E004C03E
:1016900080E090E020E030E0FA013183208308957B
:1016A00084E089BD86E089BD09B400FEFDCF80914C
:1016B000D8008F7D8093D8008091E0008260809375
:1016C000E0008091E00081FDFCCF0895CF92DF9291
:1016D000EF92FF920F931F93CF93DF93EC018B0157
:1016E0006A010E94C30C811133C0C114D10439F0C6
:1016F000F60180819181081B190BC80FD91FE12CBD
:10170000F12C0115110519F18091E80085FD16C035
:101710008091E8008E778093E800C114D10449F0ED
:10172000F60180819181E80EF91EF182E08285E068
:101730000FC00E94C30C882321F30AC089918093B3
:10174000F10001501109FFEFEF1AFF0ADACF80E034
:10175000DF91CF911F910F91FF90EF90DF90CF908D
:1017600008952091D2013091D3012617370748F010
:101770006115710539F42091E8002E772093E80077
:1017800001C0B90140E06115710591F12091CB01D3
:10179000222309F440C0253009F43FC02091E8001D
:1017A00023FD3DC02091E80022FD2FC02091E800DC
:1017B00020FFE9CF2091F20030E0FC01CF0161155C
:1017C000710559F02830310540F481918093F10082
:1017D000615071092F5F3F4FF1CF41E02830310553
:1017E00009F040E02091E8002E772093E800CBCF6D
:1017F0004111CCCF0AC08091CB01882361F08530A4
:1018000061F08091E80083FD0AC08091E80082FFCA
:10181000F2CF80E0089582E0089583E0089581E0AA
:1018200008952091D2013091D3012617370748F04F
:101830006115710539F42091E8002E772093E800B6
:1018400001C0B901FC0120E06115710579F18091B9
:10185000CB01882309F43DC0853009F43CC0809158
:10186000E80083FD3AC08091E80082FD2CC08091A1
:10187000E80080FFE9CF8091F20090E061157105EA
:1018800059F08830910540F424912093F10031966D
:10189000615071090196F2CF21E0089709F020E02C
:1018A0008091E8008E778093E800CECF2111CFCFD2
:1018B0000AC08091CB01882361F0853061F080916E
:1018C000E80083FD0AC08091E80082FFF2CF80E04B
:1018D000089582E0089583E0089581E00895982FA7
:1018E000953058F59093E900981739F07091EC0015
:1018F0002091ED005091F00003C0242F762F50E08E
:1019000021FF19C03091EB003E7F3093EB00309106
:10191000ED003D7F3093ED003091EB00316030936E
:10192000EB007093EC002093ED005093F0002091B9
:10193000EE0027FF07C09F5FD3CF8F708093E90031
:1019400081E0089580E008958091CC0187FF11C067
:101950008091E80082FD05C08091CB018111F8CF14
:1019600011C08091E8008B770BC08091CB01882358
:1019700049F08091E80080FFF8CF8091E8008E77F1
:101980008093E80008952091E4003091E50095E609
:101990004091EC00842F817040FF22C08091E800CC
:1019A00080FD1CC08091CB01882391F0853091F09F
:1019B0008091EB0085FD10C04091E4005091E5005E
:1019C0004217530729F39A01915011F784E00895C3
:1019D00082E0089583E0089581E0089580E008950D
:1019E0004091E80042FFDECF08950E94520D0E9410
:1019F000550DE0EEF0E0808181608083E8EDF0E05D
:101A000080818F77808319BCE3E6F0E0808181607C
:101A100080831092CA0108950E94520D0E94550DB4
:101A20008091D8008F778093D8008091D80080680B
:101A30008093D8008091D8008F7D8093D80084E077
:101A400089BD86E089BD09B400FEFDCF1092CB01AF
:101A50001092C7011092C9011092C80142E060E0E3
:101A600080E00E946F0C8091E1008E7F8093E10006
:101A70008091E20081608093E2008091E2008860C2
:101A80008093E2008091E0008E7F8093E0000895D3
:101A9000E3E6F0E080818E7F808381E08093CA015D
:101AA0000C940C0D1092E20008951092E10008953C
:101AB0001F920F920FB60F9211242F933F934F93C3
:101AC0005F936F937F938F939F93AF93BF93EF93A6
:101AD000FF938091E10082FF0BC08091E20082FFC2
:101AE00007C08091E1008B7F8093E1000E948B0909
:101AF0008091E10080FF19C08091E20080FF15C055
:101B00008091E2008E7F8093E2008091E20080610C
:101B10008093E2008091D80080628093D80019BC45
:101B200085E08093CB010E94930A8091E10084FFBD
:101B300030C08091E20084FF2CC084E089BD86E043
:101B400089BD09B400FEFDCF8091D8008F7D8093C0
:101B5000D8008091E1008F7E8093E1008091E200C7
:101B60008F7E8093E2008091E20081608093E200AA
:101B70008091C701882311F084E007C08091E300C1
:101B800087FD02C081E001C083E08093CB010E9409
:101B9000F20A8091E10083FF29C08091E20083FF77
:101BA00025C08091E100877F8093E10082E08093EF
:101BB000CB011092C7018091E1008E7F8093E100FC
:101BC0008091E2008E7F8093E2008091E20080614C
:101BD0008093E20042E060E080E00E946F0C809120
:101BE000F00088608093F0000E948709FF91EF91D8
:101BF000BF91AF919F918F917F916F915F914F9125
:101C00003F912F910F900FBE0F901F9018951F922C
:101C10000F920FB60F9211242F933F934F935F9320
:101C20006F937F938F939F93AF93BF93CF93DF93E4
:101C3000EF93FF93C091E900CF708091EC00D82F13
:101C4000D17080FDD0E81092E9008091F000877F8C
:101C50008093F00078940E944B0E1092E9008091DE
:101C6000F00088608093F000CD2BCF70C093E90026
:101C7000FF91EF91DF91CF91BF91AF919F918F91A4
:101C80007F916F915F914F913F912F910F900FBE78
:101C90000F901F9018951F93CF93DF93CDB7DEB7AA
:101CA000AA970FB6F894DEBF0FBECDBFECECF1E003
:101CB00088E08E0F9091F10091938E13FBCF0E94DC
:101CC000E0098091E80083FF1FC18091CC019091D1
:101CD000CD01492F50E04A30510508F015C1FA01F5
:101CE000E65CFF4F0C94AE24803881F0823809F016
:101CF0000BC18091D0018F708093E9008091EB003F
:101D000085FB882780F91092E90006C08091C80100
:101D10009091C901911182609091E800977F909312
:101D2000E8008093F1001092F100C8C0282F2D7FA9
:101D300009F0EAC0882319F0823061F0E5C0809193
:101D4000CE01813009F0E0C0933009F080E080934B
:101D5000C9012BC08091CE01811127C08091D00193
:101D60008F7009F4D1C08093E9002091EB0020FF2F
:101D70001CC0933021F48091EB00806214C09091DC
:101D8000EB0090619093EB0021E030E0A90102C0EC
:101D9000440F551F8A95E2F74093EA001092EA003B
:101DA0008091EB0088608093EB001092E9008091B5
:101DB000E800877F86C08111A7C01091CE011F77F0
:101DC0008091E3008078812B8093E3008091E8008C
:101DD000877F8093E8000E94A40C8091E80080FF38
:101DE000FCCF8091E30080688093E300111102C072
:101DF00082E001C083E08093CB0186C080588230AE
:101E000008F082C08091CE019091CF018C3D53E0CB
:101E1000950779F583E08A838AE289834FB7F8943E
:101E2000DE01139620E03EE051E2E32FF0E0509314
:101E30005700E49120FF03C0E295EF703F5FEF7021
:101E40008E2F90E0EA3010F0C79601C0C0968D93B7
:101E50009D932F5F243149F74FBF8091E800877F22
:101E60008093E8006AE270E0CE0101960E94B10B17
:101E700014C0AE014F5F5F4F6091D0010E94F80A1D
:101E8000BC01892B09F440C09091E800977F9093A2
:101E9000E80089819A810E94110C8091E8008B777B
:101EA0008093E80031C0803879F58091E800877F21
:101EB0008093E8008091C7018093F1008091E80051
:101EC0008E778093E8000E94A40C1EC081111CC074
:101ED0009091CE019230C0F48091E800877F80938A
:101EE000E8009093C7010E94A40C8091C701811162
:101EF00006C08091E30087FD02C081E001C084E05C
:101F00008093CB010E94CC098091E80083FF0AC036
:101F10008091E800877F8093E8008091EB008062E9
:101F20008093EB00AA960FB6F894DEBF0FBECDBF2C
:101F3000DF91CF911F91089590935B0180935A0197
:101F40000895E0915A01F0915B01309721F00190E2
:101F5000F081E02D099480E00895EF92FF920F93B5
:101F60001F93CF93DF93E0915A01F0915B0130977B
:101F7000B1F18C010280F381E02D09958091B601C9
:101F800082FF2DC080FF04C088E793E00E942B05EC
:101F9000E80118E082E7E82E83E0F82E8091B60190
:101FA00080FF0BC088811F928F93FF92EF920E9457
:101FB000C4050F900F900F900F90115021961111A2
:101FC000EDCF8091B60180FF0AC080E793E0DF91FA
:101FD000CF911F910F91FF90EF900C942B05DF9103
:101FE000CF911F910F91FF90EF900895E0915A01CA
:101FF000F0915B01309721F00480F581E02D099488
:10200000089520915801309159018217930771F07A
:102010009093590180935801E0915A01F0915B012E
:10202000309721F00680F781E02D099408952091E2
:102030005601309157018217930771F09093570121
:1020400080935601E0915A01F0915B01309721F0A5
:102050000084F185E02D0994089508950C942D10C5
:102060000E94E91B0C94CD05CF92DF92EF92FF9274
:102070000F931F93CF93DF9300D000D000D0CDB744
:10208000DEB70E94EA058DE5C82E81E0D82E00E07B
:1020900010E0E02E802F0E943C06F60141916F0176
:1020A000F42EF826B1F40F5F1F4F0E30110589F79B
:1020B0008FEF89838A831B820E94F21B8160782FB5
:1020C0009D838C8349815A816B818D810E94F3109D
:1020D00047C09091B60191FF04C08E830E944506CF
:1020E0008E8120E030E04F2D50E0922FBA01022E79
:1020F00002C0759567950A94E2F760FF2BC02983AB
:10210000EA8221E030E0690102C0CC0CDD1C9A9526
:10211000E2F790E08C219D21892B09F420E02B83AC
:102120000E94F21B8160782F9D838C8349815A81A4
:102130006B818D810E94F31049815A816B817C8172
:102140008D810E946C1BF801E35AFE4F8081C826E6
:10215000C08206C02F5F3F4F2830310531F6A3CF34
:102160000E946B1B0E94BF1E10915C010E94A10F78
:10217000181741F10E94A10F80935C019091B60164
:1021800092FF0EC090FF0CC01F928F938AE893E0DD
:102190009F938F930E94C4050F900F900F900F9004
:1021A00080915C0126960FB6F894DEBF0FBECDBFBE
:1021B000DF91CF911F910F91FF90EF90DF90CF9023
:1021C0000C947D1B26960FB6F894DEBF0FBECDBFD4
:1021D000DF91CF911F910F91FF90EF90DF90CF9003
:1021E00008950C948706CF93DF93CDB7DEB72B9776
:1021F0000FB6F894DEBF0FBECDBF942F4F83252FAF
:10220000588769877A878B874A855B85452B21F0BC
:102210002F3F09F59F3FF9F4DE01119686E0FD019D
:1022200011928A95E9F785E0FE01379601900D92AB
:102230008A95E1F749815A816B817C818D819E81EC
:102240000E9426182B960FB6F894DEBF0FBECDBFA6
:10225000DF91CF9108954F81588569857A858B8567
:102260000E946C1BD9CFCF93882309F4CDC0C82F0F
:10227000823859F40E94A10F81FDC6C089E30E94F3
:10228000B51A0E942E1B89E30CC0833879F40E9492
:10229000A10F80FDB9C083E50E94B51A0E942E1BD4
:1022A00083E50E94D21ACF910C942E1B843859F4E6
:1022B0000E94A10F82FDA8C087E40E94B51A0E9467
:1022C0002E1B87E4EECF8CEF8C0F813A48F48C2FD5
:1022D0000E94EB21811198C08C2F0E94B51AE3CF88
:1022E00080E28C0F883048F4C77081E001C0880F0D
:1022F000CA95EAF70E94F41AD6CF8BE58C0F83308B
:1023000078F4C53A29F0C63A31F083E890E005C088
:1023100081E890E002C082E890E0CF910C94011037
:1023200088E58C0F853108F06FC0C83A61F1C93A71
:1023300069F1CA3A71F1CB3A79F1CC3A81F1CD3AEF
:1023400089F1CE3A91F1CF3A99F1C13BA1F1C03B6D
:10235000A9F1C23BB1F1C33BB9F1C43BC1F1C53BEB
:10236000C9F1C63BD1F1C73BD9F1C83BE1F1C93B4B
:10237000E9F1CA3BF1F1CB3BF9F1CC3B09F43FC0A9
:1023800080E090E03EC082EE90E03BC089EE90E0BD
:1023900038C08AEE90E035C085EB90E032C086EB25
:1023A00090E02FC083EB90E02CC084EB90E029C03C
:1023B00087EB90E026C08CEC90E023C08DEC90E0A1
:1023C00020C083E891E01DC08AE891E01AC082E94C
:1023D00091E017C084E991E014C081E292E011C05D
:1023E00083E292E00EC084E292E00BC085E292E0CC
:1023F00008C086E292E005C087E292E002C08AE26D
:1024000092E0CF910C941710CF910895882309F48E
:102410004BC0823859F40E94A10F81FF45C089E367
:102420000E94B51A0E942E1B89E30CC0833871F4F8
:102430000E94A10F80FF38C083E50E94B51A0E9458
:102440002E1B83E50E94D21A0C942E1B843859F45B
:102450000E94A10F82FF28C087E40E94B51A0E9443
:102460002E1B87E4EFCF9CEF980F913A58F390E240
:10247000980F983050F4877091E001C0990F8A95B9
:10248000EAF7892F0E94FA1ADFCF9BE5980F933065
:1024900020F480E090E00C940110885A853120F4FB
:1024A00080E090E00C9417100895882321F00E949A
:1024B000F41A0C942E1B0895882321F00E94FA1A16
:1024C0000C942E1B0895CF92DF92EF92FF920F9300
:1024D0001F93CF93DF9300D000D000D0CDB7DEB7ED
:1024E00025E0FC01DE01119601900D922A95E1F79D
:1024F000FC0140813181F280258122952F7063811A
:102500007481672B09F4D8C23F3F19F44F3F09F497
:10251000D3C26C0149833A8389819A812E830E94B8
:10252000741A182F092F0E94731A0E948319E02F22
:10253000E295EF70F0E0EC5BFF4F2E810C94AE243F
:10254000802F807F902F9F70092F882311F0029594
:10255000007FFF2049F0002309F45FC2802F0E9412
:10256000071B0E942E1B59C2812F0E9406120023B6
:1025700009F4A2C2802F0E940D1B26960FB6F89474
:10258000DEBF0FBECDBFDF91CF911F910F91FF90A6
:10259000EF90DF90CF900C942E1B802F807F902F98
:1025A0009F70092F803211F00295007F112319F0DE
:1025B000113001F129C0FF20A9F0802F222349F119
:1025C000213039F526960FB6F894DEBF0FBECDBF89
:1025D000DF91CF911F910F91FF90EF90DF90CF90FF
:1025E0000C94171B222319F0213009F465C20E94B4
:1025F0001A1B2CC0FF20E9F0263008F05DC20E94B3
:10260000F11A802329F022C0FF20F1F0211115C01A
:10261000802F26960FB6F894DEBF0FBECDBFDF9198
:10262000CF911F910F91FF90EF90DF90CF900C947E
:102630005512253008F040C209C0F601858180FF9F
:10264000ECC18F708583E4CF2111FBC1802F69C15C
:10265000202F26952695237030E02115310521F095
:1026600021303105C9F028C2FF2021F0812F902FA1
:10267000937002C080E090E026960FB6F894DEBF1B
:102680000FBECDBFDF91CF911F910F91FF90EF90C3
:10269000DF90CF900C940110FF2021F0812F902F1C
:1026A000937002C080E090E026960FB6F894DEBFEB
:1026B0000FBECDBFDF91CF911F910F91FF90EF9093
:1026C000DF90CF900C941710812FFF2019F00E94FB
:1026D000451D02C00E94AD1D26960FB6F894DEBFC0
:1026E0000FBECDBFDF91CF911F910F91FF90EF9063
:1026F000DF90CF900C94321E802F837009F078C049
:10270000F110DAC1812F829586958770880F880F26
:10271000912F9F70C92ED12CE12CF12C082E04C0D2
:10272000CC0CDD1CEE1CFF1C0A94D2F714FF12C067
:102730004FE050E060E070E004C0440F551F661F9A
:10274000771F8A95D2F7CB01BA0160957095809575
:10275000909503C060E070E0CB01202F2695269570
:102760002370422F50E042305105D1F043305105E3
:1027700059F16C297D298E299F294130510541F15C
:1027800026960FB6F894DEBF0FBECDBFDF91CF9176
:102790001F910F91FF90EF90DF90CF900C949819BC
:1027A0006C297D298E299F2926960FB6F894DEBFC5
:1027B0000FBECDBFDF91CF911F910F91FF90EF9092
:1027C000DF90CF900C94AA190E949819C701B60106
:1027D00026960FB6F894DEBF0FBECDBFDF91CF9126
:1027E0001F910F91FF90EF90DF90CF900C9486197E
:1027F000FF2019F0802F817001C08695882309F48D
:102800005BC1812F829586958770880F880F912FE5
:102810009F70C92ED12CE12CF12C082E04C0CC0CB9
:10282000DD1CEE1CFF1C0A94D2F714FF12C04FE00F
:1028300050E060E070E004C0440F551F661F771F32
:102840008A95D2F7CB01BA016095709580959095E5
:1028500003C060E070E0CB01202F26952695237001
:10286000422F50E042305105D1F04330510559F12B
:102870006C297D298E299F294130510541F12696E9
:102880000FB6F894DEBF0FBECDBFDF91CF911F9181
:102890000F91FF90EF90DF90CF900C944F1A6C291E
:1028A0007D298E299F2926960FB6F894DEBF0FBE8C
:1028B000CDBFDF91CF911F910F91FF90EF90DF90EF
:1028C000CF900C94611A0E944F1AC701B601269648
:1028D0000FB6F894DEBF0FBECDBFDF91CF911F9131
:1028E0000F91FF90EF90DF90CF900C943D1A103F26
:1028F00041F118F4103E48F48BC0123F09F450C067
:10290000D8F1133F09F460C083C01F70802F8F710E
:10291000FF2021F00E94D619812F7BCE0E94F7194B
:10292000812F26960FB6F894DEBF0FBECDBFDF9184
:10293000CF911F910F91FF90EF90DF90CF900C946B
:102940005C12FF20A9F0253008F0B6C0802F8F71EF
:1029500026960FB6F894DEBF0FBECDBFDF91CF91A4
:102960001F910F91FF90EF90DF90CF900C941C1A65
:10297000263008F0A1C0EACFFF20A1F0802F8F7190
:1029800026960FB6F894DEBF0FBECDBFDF91CF9174
:102990001F910F91FF90EF90DF90CF900C94D6197C
:1029A000FF2061F3802F8F7126960FB6F894DEBF5B
:1029B0000FBECDBFDF91CF911F910F91FF90EF9090
:1029C000DF90CF900C94F719FF2091F0802F8F713A
:1029D00026960FB6F894DEBF0FBECDBFDF91CF9124
:1029E0001F910F91FF90EF90DF90CF900C94C11941
:1029F00026960FB6F894DEBF0FBECDBFDF91CF9104
:102A00001F910F91FF90EF90DF90CF900C94BC1925
:102A1000FF20A1F0222309F4B1CF812F26960FB613
:102A2000F894DEBF0FBECDBFDF91CF911F910F9104
:102A3000FF90EF90DF90CF900C943311222309F494
:102A4000B1CF812F26960FB6F894DEBF0FBECDBF53
:102A5000DF91CF911F910F91FF90EF90DF90CF907A
:102A60000C940612402F4F70612FC6010E94BB1CB0
:102A700026960FB6F894DEBF0FBECDBFDF91CF9183
:102A80001F910F91FF90EF90DF90CF900C94CE1894
:102A9000402F4F70612FC60126960FB6F894DEBF07
:102AA0000FBECDBFDF91CF911F910F91FF90EF909F
:102AB000DF90CF900C94BE1C26960FB6F894DEBF24
:102AC0000FBECDBFDF91CF911F910F91FF90EF907F
:102AD000DF90CF9008950E94141B0E94E31A0E9479
:102AE0002E1B0E94661F0E94321E80E090E00E9412
:102AF000011080E090E00C9417100E94041B0C94CD
:102B00006B150E94741A292F22952F7030E02C30FB
:102B100031054CF42A3031056CF422503109223051
:102B2000310588F407C02C30310549F02F303105CC
:102B300031F009C0803E48F0803F29F406C093FB85
:102B4000882780F9089580E0089581E00895CF9363
:102B5000DF9300D000D01F92CDB7DEB70F900F905B
:102B60000F900F900F90DF91CF910895CF93DF9347
:102B700000D000D000D0CDB7DEB726960FB6F894BF
:102B8000DEBF0FBECDBFDF91CF910895CF93DF930E
:102B9000C0916B0180916C01C817A1F0D0E0CE010B
:102BA00066E070E00E947D24FC01E359FE4F408105
:102BB000518162817381848195810E94B61521962D
:102BC000C770E8CFDF91CF91089540919D0150915A
:102BD0009E0160919F017091A0018091A10190914F
:102BE000A2010C94B615CF93DF938091A201829538
:102BF0008F7009F05CC080919F01882309F457C051
:102C000020916B01D0916C0140919D01C0919E017A
:102C1000E091A001F091A1012D1709F448C030E026
:102C2000309709F440C0CF3F11F44F3FE1F1C901A3
:102C300066E070E00E947D24DC01A359BE4F11962E
:102C40008C911197C8132FC08C9148132CC01296E9
:102C50008C911297811127C013968D919C91149796
:102C60008E179F0708F401978E1B9F0B883C9105D8
:102C7000D0F48091A2018F7080618093A201C9017C
:102C800066E070E00E947D24FC01EE58FE4F9081CA
:102C90009F70906190838DE991E00E946312DF91B3
:102CA000CF910C94C6152F5F3F4F2770B5CFDF91A2
:102CB000CF910895BF92CF92DF92EF92FF920F9340
:102CC0001F93CF93DF93CDB7DEB761970FB6F8941C
:102CD000DEBF0FBECDBF8C0185E0F801DE011D9681
:102CE00001900D928A95E1F7D8014C9111962C91A3
:102CF00011971296EC9012971396CD90DC90149742
:102D000050919D0160919E018091A0019091A1013F
:102D1000009709F46EC16F3F19F45F3F09F469C170
:102D2000B0909F01BB2009F4C3C03091A201C81626
:102D3000D90628F0F601E81BF90BCF0104C08095F5
:102D400090958C0D9D1DFF24F394883C910588F08F
:102D5000F12C307F09F0CBC07C2DD98AC88A522F44
:102D60006E2D89890E94A7158DE991E00E9463125A
:102D7000B4C0832F807F09F049C0621314C054137C
:102D800012C0E11010C03F7030613093A2010E9468
:102D9000E5158DE991E00E9463128091A201D801AE
:102DA00015968C9331C0CD2831F12F3F11F44F3F50
:102DB00011F1FE2CE1101FC0E0916B0130916C010C
:102DC000E31709F45CC0F0E0CF0166E070E00E9418
:102DD0007D24DC01A359BE4F11968C9111972813C5
:102DE00007C08C91481304C012968C91811103C0C6
:102DF0003196E770E5CFFE2CEE2009F416C18091E4
:102E0000A20181608093A201F12C0FC1621308C05E
:102E1000541306C0E11004C08091A201D801C1C0C2
:102E20004D872E878D859E850E9481158823E1F12F
:102E3000EE20D1F12091A201822F82958F7090E037
:102E4000029774F080919D0190919E0198878F83E5
:102E50001986DB86CA862C87CE0107960E946312EC
:102E600086E0F801ADE9B1E001900D928A95E1F7B5
:102E70000E94F3150E94E515FF24F394D6C04D87F8
:102E80002E878D859E850E94741A292F22952F707A
:102E900030E0223031050CF0BCC09F7009F0B6C0A4
:102EA000805E883008F4C1C0C8010E946312E4CF7C
:102EB000C816D90608F453C0F601E81BF90BCF0178
:102EC000883C910508F450C0F12C7C2DD98AC88A21
:102ED000522F6E2D89890E94A715EDE9F1E086E059
:102EE000DF011D928A95E9F70E94E5159EC06213E5
:102EF00014C0541312C0E11010C08091A201F80157
:102F00008583C8010E94631286E0EDE9F1E0DF01EC
:102F10001D928A95E9F7FB2C88C04D872E878D85F9
:102F20009E850E948115882309F4BECFEE2009F406
:102F3000BBCF2091A201822F82958F7090E00297E3
:102F40000CF48ECF80919D0190919E019A8389838C
:102F50001B82DD82CC822E83CE0101967FCF8095AD
:102F600090958C0D9D1DACCFFE2CEE2009F49CCFCE
:102F700062132EC054132CC02091A20120FD1FC04B
:102F8000822F82958F70D9F0D80115962C931597C2
:102F90008F3049F08F5F982F9295907F822F8F709E
:102FA000892B15968C93C8010E94631286E0F80164
:102FB000ADE9B1E001900D928A95E1F795CF86E0F9
:102FC000F801ADE9B1E001900D928A95E1F72DC0CD
:102FD0004D872E878D859E850E948115811140CF5A
:102FE0008091A20181608093A201C8010E946312B6
:102FF0001CC0EE2009F458CF4D872E878D859E8505
:103000000E948115882309F44FCF2ACF811148CF20
:103010000CC0243031050CF047CF9F7009F440CF2D
:10302000F8019581907F09F03BCF8F2D61960FB607
:10303000F894DEBF0FBECDBFDF91CF911F910F91EE
:10304000FF90EF90DF90CF90BF900895CF93DF93E4
:10305000CDB7DEB72C970FB6F894DEBF0FBECDBF4D
:103060004F83588769877A878B879C87CE0107961D
:103070000E945A16882371F08F8198852A853B8596
:10308000232B09F43FC09F3F09F068C08F3F09F030
:1030900065C038C086E0FE013796DE0111960190CA
:1030A0000D928A95E1F76F817885EA85FB853097E7
:1030B00049F17F3F11F46F3F29F180916C0190E05D
:1030C0009C012F5F3F4F2770332740916B0150E0E9
:1030D0002417350709F44BC069837A83FD83EC8399
:1030E00066E070E00E947D24DC01A359BE4F96E0AB
:1030F000FE01319601900D929A95E1F720936C01B3
:103100000E94C61580916B0190916C018917E9F1BD
:1031100090E066E070E00E947D2483599E4F0E94FB
:103120005A16882391F180916B0190E066E070E07F
:103130000E947D24FC01E359FE4F40815181628150
:103140007381848195810E94B61580916B0190E016
:1031500001968770992780936B01D4CF4F81588552
:1031600069857A858B859C850E94B615CBCF0E9498
:103170007D1510926C0110926B01EDE9F1E086E093
:10318000DF011D928A95E9F7BDCF2C960FB6F89412
:10319000DEBF0FBECDBFDF91CF910895DF92EF92DA
:1031A000FF920F931F93CF93DF93FC01892B09F4B8
:1031B0008AC0E12CF12CDD24D394EF012196849177
:1031C000853709F461C058F4843708F04EC0843064
:1031D00008F06AC08130D1F0823071F174C0883754
:1031E00009F45DC050F4863709F455C0873709F0FB
:1031F0006AC08E2D0E94011B54C09CE7980F903727
:1032000008F061C08F770E94061250C08F010E5FD8
:103210001F4FFE01849190E2980F983050F4877010
:10322000FD2D01C0FF0F8A95EAF78F2F0E94071B23
:1032300014C00E94331113C08F010E5F1F4FFE0197
:10324000C49180E28C0F883060F4C7708D2D01C06E
:10325000880FCA95EAF70E940D1B0E942E1BE801F9
:1032600025C08C2F0E940612FACF9F012E5F3F4F80
:10327000FE01C491CC2369F08FE99FE00197F1F73B
:1032800000C00000C150F6CF9F012E5F3F4FFE01EE
:10329000F490E9010BC00E94F11AE82E07C00E94C9
:1032A000041B0E942E1B02C00E9433118F2D882305
:1032B00041F0EFE9FFE03197F1F700C000008150E5
:1032C000F6CFFE017ACFDF91CF911F910F91FF9042
:1032D000EF90DF9008956093A7017093A801809309
:1032E000A9019093AA010E947B1B0C946B1560931B
:1032F000A3017093A4018093A5019093A6010E945D
:103300007C1B0C946B1508950C946B190F931F93F1
:103310000091A7011091A8012091A9013091AA0163
:10332000602B712B822B932B1F910F910C946B1997
:103330000F931F930091A7011091A8012091A9015B
:103340003091AA0160237123822393231F910F914F
:103350000C946B190F931F930091A7011091A80172
:103360002091A9013091AA01602771278227932714
:103370001F910F910C946B1960E070E0CB010C94DD
:1033800077190F931F9341E050E060E070E08A01ED
:103390009B0104C0000F111F221F331F8A95D2F713
:1033A000C901B8011F910F910C9477190F931F93C6
:1033B00041E050E060E070E004C0440F551F661F1C
:1033C000771F8A95D2F78091A3019091A401A091D3
:1033D000A501B091A6018A019B01082B192B2A2B6C
:1033E0003B2BC901B8011F910F910C9477190F93D2
:1033F0001F9341E050E060E070E004C0440F551FAF
:10340000661F771F8A95D2F7409550956095709505
:103410008091A3019091A401A091A501B091A60172
:103420008A019B01082319232A233B23C901B801E0
:103430001F910F910C9477190F931F9341E050E067
:1034400060E070E004C0440F551F661F771F8A9527
:10345000D2F78091A3019091A401A091A501B09110
:10346000A6018A019B01082719272A273B27C901A2
:10347000B8011F910F910C9477190F931F9300912E
:10348000A3011091A4012091A5013091A601602B08
:10349000712B822B932B1F910F910C9477190F9303
:1034A0001F930091A3011091A4012091A5013091D7
:1034B000A60160237123822393231F910F910C9403
:1034C00077190F931F930091A3011091A4012091EC
:1034D000A5013091A60160277127822793271F91AC
:1034E0000F910C9477190895CF92DF92EF92FF928B
:1034F0000F931F93CF93DF938C01C090A701D090BF
:10350000A801E090A901F090AA014091A301509177
:10351000A4016091A5017091A601C42AD52AE62ACA
:10352000F72ACFE1D0E0D701C6010C2E04C0B69532
:10353000A795979587950A94D2F780FF07C0B801A1
:103540008C2F0E948C1C8130910531F4219758F703
:10355000B80180E00E948C1CDF91CF911F910F91E8
:10356000FF90EF90DF90CF90089520910B01309164
:103570000C01F90132969FEF40E05191581789F004
:103580009F3F19F4511101C0942F4F5F4630A9F7A6
:103590009F3F39F0F901E90FF11D97FDFA958283FC
:1035A0000895089520910B0130910C01F901329694
:1035B000285F3F4F9081981301C010823196E21727
:1035C000F307C1F7089581E090E0E0910B01F091DD
:1035D0000C01E80FF91F1082019688309105A9F7B8
:1035E00008958091B50108959091B501892B80933C
:1035F000B501089580959091B50189238093B50117
:1036000008958093B50108951092B50108959091A1
:10361000B401892B8093B401089580959091B401F1
:1036200089238093B40108951092B4010895809382
:10363000AB0108951092AB01089580910B01909118
:103640000C01FC0131969C01285F3F4F80E0919175
:1036500091118F5FE217F307D1F70895E0910B0105
:10366000F0910C018091B5018083E0910B01F09104
:103670000C0190818091B401892B80838091AB01F2
:10368000882361F0E0910B01F0910C019081892B6E
:1036900080830E941D1B81111092AB0180910B0150
:1036A00090910C010C94AD0F9093330180933201F3
:1036B00008958295982F9C7C292F26952695982FE2
:1036C0009373990F990F922B892F8A7A8695957506
:1036D000990F892B08950895CF93DF9300D000D0E0
:1036E0001F92CDB7DEB70F900F900F900F900F90F5
:1036F000DF91CF910895089508950C94F110809171
:10370000CB01843021F11092B70120E488E190E0F0
:103710000FB6F894A895809360000FBE20936000C8
:1037200083B7817F846083BF83B7816083BF7894D0
:10373000889583B78E7F83BF0FB6F894A895809144
:103740006000886180936000109260000FBE089551
:1037500008950895CF930E94A81B0E94EA050E9435
:10376000A91BC0E08C2F0E943C06811104C0CF5FD2
:10377000CE30C1F701C081E0CF9108950C947D1542
:103780001F920F920FB60F9211248F939F93AF93B6
:10379000BF938091B701811113C08091B8019091BE
:1037A000B901A091BA01B091BB014196A11DB11D13
:1037B0008093B8019093B901A093BA01B093BB0173
:1037C000BF91AF919F918F910F900FBE0F901F905F
:1037D000189582E084BD93E095BD9AEF97BD8093E4
:1037E0006E0008952FB7F8948091B8019091B901B7
:1037F000A091BA01B091BB012FBF08952FB7F894E3
:103800006091B8017091B9018091BA019091BB01AA
:103810002FBF0895CF92DF92EF92FF920F931F93E5
:103820002FB7F8944091B8015091B9016091BA0155
:103830007091BB012FBF6A017B01EE24FF248C0134
:1038400020E030E0C016D106E206F30610F4415045
:1038500051099A01281B390BC9011F910F91FF9043
:10386000EF90DF90CF9008951F920F920FB60F92B6
:1038700011248F939F93AF93BF938091B801909140
:10388000B901A091BA01B091BB010196A11DB11D72
:103890008093B8019093B901A093BA01B093BB0192
:1038A000BF91AF919F918F910F900FBE0F901F907E
:1038B00018950E94F50CF8942FEF87EA91E62150B5
:1038C00080409040E1F700C0000087E090EBDC0111
:1038D0008093D4019093D501A093D601B093D701E2
:1038E0009CE088E10FB6F894A895809360000FBE25
:1038F00090936000FFCFE92FF0E093E0EE0FFF1F01
:103900009A95E1F7E80FF11DE855FF4F9491892F43
:103910008F7092959F700895CF93C82FCB010E940E
:103920007B1C492F90E0242F30E054E0220F331FFE
:103930005A95E1F7282B392B2038310519F480E00E
:1039400090E017C0EC2FF0E023E0EE0FFF1F2A9568
:10395000E1F74770E40FF11D34E0EE0FFF1F3A95D9
:10396000E1F7E80FF91FEE0FFF1FE050F8498591CE
:103970009491CF91089580E090E00895089580910A
:10398000BE0180FF0CC08091100190E065E070E006
:103990000E947D2495958795959587952EC081FFEA
:1039A0000AC08091100190E065E070E00E947D24E3
:1039B0009595879522C082FF08C08091100190E004
:1039C00065E070E00E947D2418C02091BF01222391
:1039D000D1F030910F01231780F78091100190E012
:1039E00065E070E00E947D24622F70E00E947D24DB
:1039F000632F70E00E949A24CB018038910530F447
:103A0000009731F0089585E090E008958FE70895DC
:103A100081E008958091BE0180FF08C060910E0191
:103A200070E0759567957595679523C081FF06C011
:103A300060910E0170E0759567951BC082FF04C010
:103A400060910E0170E012C06091BF016623D1F059
:103A500020910D016217A0F780910E0170E090E0B7
:103A60000E947D24622F70E00E949A2460387105C4
:103A700028F46115710521F0862F08958FE70895C8
:103A800081E0089561E070E0F4CF803F21F40E946E
:103A9000BF1C819504C0813F29F40E94BF1C809304
:103AA000C2010895823F21F40E94BF1C819504C089
:103AB000833F29F40E94BF1C8093C1010895893F70
:103AC00019F40E940A1D05C08A3F31F40E940A1DA4
:103AD00081958093C30108958B3F21F40E940A1DB4
:103AE000819504C08C3F29F40E940A1D8093C40173
:103AF0000895843F21F48091C001816017C0853F03
:103B000021F48091C001826011C0863F21F4809130
:103B1000C00184600BC0873F21F48091C0018860A0
:103B200005C0883F31F48091C00180618093C0015D
:103B300008958D3F21F48091BE0181600BC08E3FBE
:103B400021F48091BE01826005C08F3F29F48091ED
:103B5000BE0184608093BE010895803F39F4809156
:103B6000C20187FF6CC01092C20169C0813F29F475
:103B70008091C2011816BCF362C09091C101823FCE
:103B800029F497FF5CC01092C10159C0833F19F41A
:103B90001916CCF354C0893F41F48091C301181623
:103BA0000CF04DC01092C3014AC08A3F29F48091A5
:103BB000C30187FF44C0F6CF8B3F39F48091C40125
:103BC00087FF3DC01092C4013AC08C3F29F4809118
:103BD000C4011816BCF333C0843F21F48091C001A6
:103BE0008E7F17C0853F21F48091C0018D7F11C069
:103BF000863F21F48091C0018B7F0BC0873F21F469
:103C00008091C001877F05C0883F31F48091C00159
:103C10008F7E8093C00113C08D3F21F48091BE013F
:103C20008E7F0BC08E3F21F48091BE018D7F05C039
:103C30008F3F29F48091BE018B7F8093BE018091DC
:103C4000C10181110EC08091C20181110AC0809111
:103C5000C301811106C08091C401811102C010927C
:103C6000BF0108958091B60183FF7EC08CEB93E085
:103C70000E942B058091C0011F928F9387EB93E0E8
:103C80009F938F930E94C40585EB93E00E942B05C0
:103C90008091C101282F082E000C330B3F938F9386
:103CA00082EB93E09F938F930E94C40580EB93E097
:103CB0000E942B058091C201282F082E000C330B87
:103CC0003F938F938DEA93E09F938F930E94C40557
:103CD0008BEA93E00E942B058091C301282F082EC8
:103CE000000C330B3F938F9388EA93E09F938F935D
:103CF0000E94C40586EA93E00E942B058091C401CE
:103D0000282F082E000C330B3F938F9383EA93E008
:103D10009F938F930E94C40580EA93E00E942B0535
:103D20008091BF011F928F938DE993E09F938F93B2
:103D30000E94C4058BE993E00E942B058091BE018F
:103D40001F928F9388E993E09F938F930E94C405FD
:103D500085E993E00E942B058DB79EB74C960FB670
:103D6000F8949EBF0FBE8DBF80EC91E00E94F60FCD
:103D70000E94F21B9093BD018093BC0108951F9394
:103D8000CF93DF938091BC019091BD010E940A1CEA
:103D9000FC012091BF01222329F090911101892F6C
:103DA00090E007C08091120190E06AE070E00E940C
:103DB0007D24E817F90708F485C08091C101C091FE
:103DC000C201D091C3011091C401811107C0C1117A
:103DD00075C0D11173C0111171C074C02F3F19F09B
:103DE0002F5F2093BF01181624F40E94BF1C8093FC
:103DF000C1018091C10187FF05C00E94BF1C819550
:103E00008093C1011C1624F40E94BF1C8093C20140
:103E10008091C20187FF05C00E94BF1C81958093DD
:103E2000C2016091C101662331F1C091C201CC236E
:103E300011F1062E000C770B880B990B0E947C2346
:103E400023E333E343E35FE30E94E0230E94442340
:103E50006093C1016C2FCC0F770B880B990B0E94DC
:103E60007C2323E333E343E35FE30E94E0230E94E8
:103E700044236093C2011D1624F40E940A1D8093FE
:103E8000C3018091C30187FF05C00E940A1D81956F
:103E90008093C301111624F40E940A1D8093C4016B
:103EA0008091C40187FF05C00E940A1D81958093FF
:103EB000C401DF91CF911F910C94321E2F3F09F066
:103EC0008FCF97CFDF91CF911F910895E0ECF1E074
:103ED00085E0DF011D928A95E9F71092BF011092EB
:103EE000BE0108958FED95E00E942B051F9281E0A1
:103EF0008F931F9285E08F9381E995E09F938F9335
:103F00000E94C4050F900F900F900F900F900F908C
:103F100008958330E9F128F4813061F0823009F1AD
:103F20000895853009F462C008F449C0863009F468
:103F300074C0089580911201262F30E0280F311DA2
:103F40002F3F310524F4680F6093120103C08FEFF7
:103F500080931201809112011F928F938AEC94E05A
:103F600072C080911101262F30E0280F311D2F3FA4
:103F7000310524F4680F6093110103C08FEF809323
:103F80001101809111011F928F9388EB94E05BC027
:103F900080911001262F30E0280F311D2F3F310571
:103FA00024F4680F6093100103C08FEF8093100119
:103FB000809110011F928F9385EA94E044C0809114
:103FC0000F01262F30E0280F311D2F3F310524F43B
:103FD000680F60930F0103C08FEF80930F018091F2
:103FE0000F011F928F9380E994E02DC080910E0104
:103FF000262F30E0280F311D2F3F310524F4680FA4
:1040000060930E0103C08FEF80930E0180910E012B
:104010001F928F9387E794E016C080910D01262FA1
:1040200030E0280F311D2F3F310524F4680F6093D5
:104030000D0103C08FEF80930D0180910D011F9240
:104040008F938CE594E09F938F930E94C4050F900B
:104050000F900F900F900895833081F128F48130F4
:1040600059F08230D1F00895853009F449C0B8F193
:10407000863009F456C0089580911201681720F423
:10408000861B8093120102C01092120180911201CE
:104090001F928F938DE494E054C0809111016817B2
:1040A00020F4861B8093110102C0109211018091AF
:1040B00011011F928F938BE394E043C08091100114
:1040C000681720F4861B8093100102C01092100123
:1040D000809110011F928F9388E294E032C080910A
:1040E0000F01681720F4861B80930F0102C0109205
:1040F0000F0180910F011F928F9383E194E021C003
:1041000080910E01681720F4861B80930E0102C077
:1041100010920E0180910E011F928F938AEF93E00F
:1041200010C080910D01681720F4861B80930D014B
:1041300002C010920D0180910D011F928F938FED9F
:1041400093E09F938F930E94C4050F900F900F9060
:104150000F900895CF93C82F1F928F9384EE96E00F
:104160009F938F930E94C40581E090E0A0E0B0E0AF
:10417000BC01CD0104C0660F771F881F991FCA9527
:10418000D2F70E9484190F900F900F900F90CF914B
:104190000C947D15CF93873288F58E3108F00BC1D2
:1041A0008E3009F487C0D8F4873009F460C08B30B2
:1041B00009F44FC0863009F002C18091B601817FB9
:1041C0008E7F8093B60189EE96E00E942B0587EAE8
:1041D00099E00E942B0581E08093C60146C086319C
:1041E00009F4B0C020F4803109F47AC0E8C0893104
:1041F00009F491C08B3109F449C0E1C0883349F119
:1042000050F4893209F4D5C0853309F4D2C087321D
:1042100009F0D5C0CEC0833409F4CBC028F48A336A
:1042200008F4CDC08953C8C0883409F0C8C00E94C2
:104230007D1586E999E00E942B052FEF83ED90E331
:10424000215080409040E1F700C000000E94591CBE
:104250000CC080E197E041C08DE799E00E942B05FA
:104260008091B60181608093B601C1E0ADC08091BC
:10427000B601C82FC17080FFEFCF89E899E00E9496
:104280002B058091B601817F8E7F3FC09091B60152
:1042900091FBCC27C0F981E0C827892FC0FB81F9A9
:1042A0008093B601CC2319F080E799E029C082E61B
:1042B00099E013C09091B60192FBCC27C0F981E040
:1042C000C827892FC0FB82F98093B601CC2319F04F
:1042D00083E599E015C083E499E00E942B05C5CFE2
:1042E0009091B60193FBCC27C0F981E0C827892FB4
:1042F000C0FB83F98093B601CC2351F087E399E0AA
:104300000E942B058091B60181608093B6015CC04C
:104310008AE299E0E2CF8BE199E00E942B0586EFDB
:1043200098E00E942B058FEA98E00E942B0582E816
:1043300098E00E942B058DE398E00E942B058EE00B
:1043400098E0CBCF80E098E00E942B050E94A10F5F
:104350001F928F9386EE97E09F938F930E94C405E0
:1043600080910A011F928F938FEC97E09F938F9318
:104370000E94C405809155011F928F938CEB97E0AA
:104380009F938F930E94C4050E94FE1B9F938F935F
:104390007F936F9385EA97E09F938F930E94C40564
:1043A0008DB79EB742960FB6F8949EBF0FBE8DBFD5
:1043B0005CCF80E001C08D510E94AA2056CF83EAD5
:1043C00097E00E942B05C0E08C2FCF91089580E0EC
:1043D000089580E00895CF93C82F8091C601813061
:1043E00081F020F0823009F44FC046C1E0910B010A
:1043F000F0910C0180818E3069F0873009F03EC168
:1044000009C0E0910B01F0910C0180818E3011F018
:10441000873061F48C2F0E94E721811104C08C2F1A
:104420000E94CA202FC081E090E02CC08C2F0E94F7
:10443000E921811126C0C431E1F070F4CB3081F064
:10444000C031D1F40E94721F8CED96E00E942B05C2
:1044500082E08093C60115C0C93259F0C83361F4B7
:1044600089EE96E00E942B0580EE96E00E942B05D7
:1044700008C01092C60104C18AED96E00E942B0587
:10448000FFC081E08170FEC0C43228F5CE3108F053
:10449000C1C0CB30A1F1D0F4C73009F0D3C08EE158
:1044A0008093120182E3809311018AE080931001CE
:1044B00084E180930F0188E080930E0188E280936D
:1044C0000D0180E895E00E942B05BFC0C33149F182
:1044D000C431C1F0B7C0CB3409F4A9C028F4C93243
:1044E00089F0C83361F0AEC0C13509F49EC0C23551
:1044F00009F499C0CE3409F0A5C06AE09EC00E94BC
:10450000721FA3C08091C501882319F01092C501C4
:104510009CC08DE895E00E942B0581E08093C60148
:10452000B1C087E695E00E942B0585E595E00E94E5
:104530002B05809112011F928F9382E595E09F9346
:104540008F930E94C40580E595E00E942B058EE3C1
:1045500095E00E942B05809111011F928F938BE3B0
:1045600095E09F938F930E94C40589E395E00E9494
:104570002B058AE295E00E942B05809110011F9285
:104580008F9387E295E09F938F930E94C40585E205
:1045900095E00E942B0584E195E00E942B05809117
:1045A0000F011F928F9381E195E09F938F930E945B
:1045B000C4058FE095E00E942B058AEF94E00E94ED
:1045C0002B0580910E011F928F9387EF94E09F93AC
:1045D0008F930E94C40585EF94E00E942B058EED19
:1045E00094E00E942B0580910D011F928F938BED1B
:1045F00094E09F938F930E94C40589ED94E00E94FC
:104600002B058DB79EB748960FB6F8949EBF0FBE88
:104610008DBF1BC0CE51EC2FF0E0E95DFE4F8081D5
:104620008093C50112C061E003C061E006C06AE08A
:104630008091C5010E94891F08C08091C5010E9418
:104640002C2003C08EE795E013C08091C50188231C
:1046500069F01F928F9388E795E09F938F930E9454
:10466000C4050F900F900F900F9004C085E795E060
:104670000E942B0581E006C01092C60180E002C0B6
:1046800080E000CFCF9108950E944B236894B11130
:104690000C94DA2308950E94BF2388F09F5798F066
:1046A000B92F9927B751B0F0E1F0660F771F881F37
:1046B000991F1AF0BA95C9F714C0B13091F00E9451
:1046C000D923B1E008950C94D923672F782F882738
:1046D000B85F39F0B93FCCF3869577956795B39578
:1046E000D9F73EF490958095709561957F4F8F4FE7
:1046F0009F4F0895E89409C097FB3EF490958095EC
:10470000709561957F4F8F4F9F4F9923A9F0F92F97
:1047100096E9BB279395F695879577956795B79515
:10472000F111F8CFFAF4BB0F11F460FF1BC06F5FFB
:104730007F4F8F4F9F4F16C0882311F096E911C00D
:10474000772321F09EE8872F762F05C0662371F02E
:1047500096E8862F70E060E02AF09A95660F771F42
:10476000881FDAF7880F9695879597F9089557FD72
:104770009058440F551F59F05F3F71F04795880FCF
:1047800097FB991F61F09F3F79F087950895121666
:1047900013061406551FF2CF4695F1DF08C0161612
:1047A00017061806991FF1CF8695710561050894C3
:1047B0000895E894BB2766277727CB0197F90895DA
:1047C0000E94F2230C946C240E945E2438F00E9414
:1047D000652420F0952311F00C9455240C945B244F
:1047E0000C94DA230E94B72378F39923C9F3552355
:1047F000B9F3950F50E0551FAA27EE27FF27BB27D7
:1048000000240894679520F4E20FF31FB41F0A1EDA
:10481000220F331F441FAA1F6695A9F7779530F41E
:10482000F30FB41F0A1E121E08F46395330F441FC2
:10483000AA1F221F769599F7879520F4B40F0A1EB8
:10484000121E631F440FAA1F221F331F8695A9F74C
:10485000862F712D602D11249F5750409AF0F1F052
:1048600088234AF0EE0FFF1FBB1F661F771F881FAC
:1048700091505040A9F79E3F510580F00C9455246B
:104880000C94DA235F3FE4F3983ED4F38695779552
:104890006795B795F795E7959F5FC1F7FE2B880F52
:1048A000911D9695879597F9089597F99F6780E8E8
:1048B00070E060E008959FEF80EC089500240A9472
:1048C0001616170618060906089500240A941216EB
:1048D0001306140605060895092E0394000C11F41E
:1048E000882352F0BB0F40F4BF2B11F460FF04C0CB
:1048F0006F5F7F4F8F4F9F4F08950024552704C04F
:10490000080E591F880F991F009729F07695679513
:10491000B8F37105B9F7802D952F0895991B79E0AB
:1049200004C0991F961708F0961B881F7A95C9F73F
:104930008095089597FB072E16F4009407D077FD15
:1049400009D00E94B42407FC05D03EF490958195CF
:104950009F4F0895709561957F4F0895EE0FFF1F4B
:104960000590F491E02D0994AA1BBB1B51E107C0EF
:10497000AA1FBB1FA617B70710F0A61BB70B881FEF
:10498000991F5A95A9F780959095BC01CD0108957E
:04499000F894FFCFC9
:104994006608570934090009CC0801AC0128081439
:1049A4000A321E404D36223003E302AD028B021759
:1049B40002300249026202010203040506070809E3
:0249C4000000F1
:106800000000000000000000040005000600070072
:10681000080009000A000B000C000D000E000F001C
:1068200010001100120013001400150016001700CC
:10683000180019001A001B001C001D001E001F007C
:10684000200021002200230024002500260027002C
:10685000280000002A002B002C002D002E002F0005
:10686000300031A1320033003400350036003700EB
:106870003800E00000000000000000000000000000
:106880000000000000000000000000000000000008
:1068900000000000000000000000000000004F00A9
:1068A000500051005200530067005400550056003C
:1068B000580059005A005B005C005D005E005F00FC
:1068C0006000610062006300640000005700000087
:1068D00000000000000000000000000000000000B8
:1068E00000000000000000000000000000000000A8
:1068F0000000E100E200E300000000000000F1A160
:106900000100010001000100EA4401000100E2442D
:106910000100010001000100460001004A004B0097
:10692000010001004700480001000100E9440100A6
:106930000100010001000100010001003A003B00DC
:106940003C003D003E003F0040004100420043004B
:10695000010000004C00010001004400450052000D
:1069600049000100010050004F0029004D004E0079
:1069700051000100010001000100010001000100BF
:1069800001000100010001000100010001000100FF
:1069900001000100010001000100010001004D00A3
:1069A0004A004E004B0001000100010001000100FF
:1069B00001000100010001000100010001000100CF
:1069C00001000100010001000100010001000100BF
:1069D00001000100010001000100010001000100AF
:1069E000010001000100010001000100010001009F
:1069F000010001000100010001000100010001008F
:00000001FF
